:020000040800F2
:1000000000090020B5040008D52500088D2500084A
:10001000B52500088D250008AD250008B7040008A7
:10002000B7040008B7040008B7040008C935000881
:10003000B7040008B7040008B70400087D430008AF
:10004000B7040008B7040008B7040008B7040008A4
:10005000B7040008B7040008614000088D4000089C
:10006000B9400008E540000811410008B704000845
:10007000B7040008B7040008B7040008B704000874
:10008000B7040008B7040008B704000841250008B9
:100090006D2500087D250008B70400083D410008D3
:1000A000B7040008B7040008B7040008B704000844
:1000B000B7040008B7040008B7040008B704000834
:1000C000B7040008B7040008B7040008B704000824
:1000D000B70400086D45000881450008B704000812
:1000E000A5410008B7040008B7040008B7040008D9
:1000F000B7040008B7040008B7040008B7040008F4
:10010000B7040008B7040008B7040008B7040008E3
:10011000B7040008B7040008B7040008B7040008D3
:10012000B7040008B7040008B7040008B7040008C3
:10013000B7040008B7040008B7040008B7040008B3
:10014000B7040008B7040008B7040008B7040008A3
:10015000B7040008B7040008B7040008B704000893
:10016000B7040008B7040008B7040008B704000883
:10017000B7040008B7040008B7040008B704000873
:10018000B7040008B7040008B7040008B704000863
:10019000B7040008B7040008B7040008B704000853
:1001A000291200080000000000000000000000000C
:1001B00053B94AB9002908BF00281CBF4FF0FF31CE
:1001C0004FF0FF3000F074B9ADF1080C6DE904CECA
:1001D00000F006F8DDF804E0DDE9022304B0704722
:1001E0002DE9F047089D04468E46002B4DD18A42EA
:1001F000944669D9B2FA82F252B101FA02F3C2F11D
:10020000200120FA01F10CFA02FC41EA030E9440AD
:100210004FEA1C48210CBEFBF8F61FFA8CF708FBCE
:1002200016E341EA034306FB07F199420AD91CEBA6
:10023000030306F1FF3080F01F81994240F21C81D8
:10024000023E63445B1AA4B2B3FBF8F008FB103320
:1002500044EA034400FB07F7A7420AD91CEB040455
:1002600000F1FF3380F00A81A74240F20781644425
:10027000023840EA0640E41B00261DB1D4400023AA
:10028000C5E900433146BDE8F0878B4209D9002D0E
:1002900000F0EF800026C5E9000130463146BDE898
:1002A000F087B3FA83F6002E4AD18B4202D3824202
:1002B00000F2F980841A61EB030301209E46002DB1
:1002C000E0D0C5E9004EDDE702B9FFDEB2FA82F206
:1002D000002A40F09280A1EB0C014FEA1C471FFA64
:1002E0008CFE0126200CB1FBF7F307FB131140EA4B
:1002F00001410EFB03F0884208D91CEB010103F118
:10030000FF3802D2884200F2CB804346091AA4B2D9
:10031000B1FBF7F007FB101144EA01440EFB00FEAD
:10032000A64508D91CEB040400F1FF3102D2A64512
:1003300000F2BB800846A4EB0E0440EA03409CE7B1
:10034000C6F12007B34022FA07FC4CEA030C20FA5E
:1003500007F401FA06F31C43F9404FEA1C4900FA7E
:1003600006F3B1FBF9F8200C1FFA8CFE09FB1811FB
:1003700040EA014108FB0EF0884202FA06F20BD96E
:100380001CEB010108F1FF3A80F08880884240F2BE
:100390008580A8F102086144091AA4B2B1FBF9F002
:1003A00009FB101144EA014100FB0EFE8E4508D9FD
:1003B0001CEB010100F1FF346CD28E456AD9023882
:1003C000614440EA0840A0FB0294A1EB0E01A14267
:1003D000C846A64656D353D05DB1B3EB080261EBD5
:1003E0000E0101FA07F722FA06F3F1401F43C5E9AF
:1003F000007100263146BDE8F087C2F12003D840E5
:100400000CFA02FC21FA03F3914001434FEA1C4726
:100410001FFA8CFEB3FBF7F007FB10360B0C43EA18
:10042000064300FB0EF69E4204FA02F408D91CEBC8
:10043000030300F1FF382FD29E422DD902386344C6
:100440009B1B89B2B3FBF7F607FB163341EA034166
:1004500006FB0EF38B4208D91CEB010106F1FF38B5
:1004600016D28B4214D9023E6144C91A46EA0046AC
:1004700038E72E46284605E70646E3E61846F8E63E
:100480004B45A9D2B9EB020864EB0C0E0138A3E787
:100490004646EAE7204694E74046D1E7D0467BE768
:1004A000023B614432E7304609E76444023842E7E0
:1004B000704700BF02E000F000F8FEE772B6374870
:1004C00080F30888364880F3098836483649086042
:1004D00040F20000CCF200004EF63471CEF2000182
:1004E0000860BFF34F8FBFF36F8F40F20000C0F280
:1004F000F0004EF68851CEF200010860BFF34F8F36
:10050000BFF36F8F4FF00000E1EE100A4EF63C7122
:10051000CEF200010860062080F31488BFF36F8FCD
:1005200003F052FC03F0C6FC4FF055301F491B4A44
:1005300091423CBF41F8040BFAE71D49184A914229
:100540003CBF41F8040BFAE71A491B4A1B4B9A427D
:100550003EBF51F8040B42F8040BF8E7002018499D
:10056000184A91423CBF41F8040BFAE703F030FC13
:1005700003F0DCFC144C154DAC4203DA54F8041BB8
:100580008847F9E700F042F8114C124DAC4203DA0B
:1005900054F8041B8847F9E703F018BC0009002051
:1005A000001100200000000808ED00E0000100201C
:1005B00000090020784B0008001100207C11002069
:1005C00080110020583C0020A0010008A401000870
:1005D000A4010008A40100082DE9F04F2DED108AB8
:1005E000C1F80CD0C3689D46BDEC108ABDE8F08F01
:1005F000002383F311882846A047002003F06EF9FA
:10060000FEE703F0D1F800DFFEE70000F8B500F0E8
:100610001DFE03F07DFB074603F0CCFB05460028DA
:1006200040D12C4B9F423DD001339F423DD02A4BBD
:1006300027F0FF029A423BD1F8B200F043FC2E466D
:1006400042F2107400F044FC08B10024264601F088
:10065000B5F888B3032000F045F80024264635B1EC
:100660001E4B9F4203D003F09DFB00242646002032
:1006700003F058FB1A4B1B6913F0400322D00EB154
:1006800000F046F800F056FC00F0E2FD01F0AAFF91
:100690000546CCB101F0A6FF401BA04214D900F0E2
:1006A00037F8F3E72E460024CCE704460126C9E7D5
:1006B00006464FF47A74C5E7002CD0D04FF47A7414
:1006C0000126CCE71C46DDE700F07CFC012003F0AE
:1006D0000BF9DEE7010007B0000008B0263A09B0C8
:1006E00000040048084B187003280CD8DFE800F01D
:1006F00008050208022000F007BE022000F0FCBD41
:10070000024B00225A6070478011002084110020A3
:1007100038B501F053F830B11F4B03221A701F4B4C
:1007200000225A6038BD1E4B1E4A19680131F9D0AB
:1007300004339342F9D11C4C194DD4F80428AA4231
:10074000F0D31A4B9B6803F1006303F5D0439A4240
:10075000E8D203F0FBFA03F00DFB002000F092FD5D
:100760000220FFF7BFFF124BDA690022DA61D96974
:1007700099699A619B6972B64FF0E0233021C3F802
:10078000085DD4F80038D4F8042881F311889D4618
:1007900083F308881047C5E78011002084110020EA
:1007A00000680008206800080060000800110020B0
:1007B00000100240094A136849F2690099B21B0C03
:1007C00000FB01331360064B186844F2506182B29B
:1007D000000C01FB0200186080B270471411002069
:1007E0001011002010B500211022044600F0A6FDD3
:1007F000034B03CB206061601868A06010BD00BF90
:10080000ACF7FF1F2DE9F041ADF54E7D0DF1340839
:100810006CAC40F2751207460D460EA80021C8F8D0
:10082000001000F08BFD4FF4C4720021204600F050
:1008300085FD01F0D7FE274B4FF47A72B0FBF2F042
:10084000186093E80700022384E807000DF5E970BB
:100850002382FFF7C7FF4EF603431F49238406A8F0
:1008600004F0BAF81B2384F832310DF2E32206AB10
:100870000DF1300C1E4603CE6645106051603346C4
:1008800002F10802F6D13188B378937011802046C6
:100890004146012200F09EFD00230393AB7E0293AC
:1008A00005F11903019380B20123CDE9048000937F
:1008B000E97E06A3D3E90023384602F05BFA0DF582
:1008C0004E7DBDE8F08100BFAFF300809E6AC42179
:1008D000818A46EE8C110020E84900082DE9F0419C
:1008E0002C4C237ADAB080460D465BBB27A92846FC
:1008F00000F080FE0746002842D19DF89D60C82E7A
:100900003ED801464FF4A662204600F017FD4FF492
:100910008073C4F8F8314FF40073C4F80C334FF40B
:100920004073C4F8203432460DF19E0104F10900F1
:1009300000F0F2FC26449DF89C30777223720BB9CC
:10094000EB7E23728122002106AC27A800F0F6FC82
:100950000122214627A800F089FE00230393AB7EE5
:10096000029305F1190380B201932823CDE90440D5
:100970000093E97E05A3D3E90023404602F0FAF98B
:100980005AB0BDE8F08100BFAFF30080264172721B
:10099000DF25D7B7A8320020F0B5254E4FF48A7571
:1009A00005FB0065F1B096F8D83085F8DC300024FE
:1009B000D822214685F8E8403AA800F0BFFC06F1AD
:1009C000090000F0B3FCD5F8E4308DF8F000C2B2B5
:1009D00006AF06F109010DF1F100CDE93A3400F05E
:1009E0009BFC394601223AA800F06CFE80B2CDE9AA
:1009F000047008230127CDE9023706F1D8030193DB
:100A000030230093317A0B4807A3D3E9002302F087
:100A1000B1F9A04206DD01F0E5FDC5F8E000384679
:100A200071B0F0BD2046FBE778F6339F93CACD8DB9
:100A3000A8320020A42100202DE9F0411D4D1E4EBA
:100A40001E4F86B0284602F0C1F9034658B3002471
:100A5000CDE90344ADF81440027B8DF81420996869
:100A60004068029403AA03C21B68DFF8548043F075
:100A70000043029301F0B8FD821941F10003009494
:100A800002A9384601F07CF8A04205DD284602F0B4
:100A9000A1F988F80040D5E798F80030072B05D871
:100AA000013388F8003006B0BDE8F081014802F05B
:100AB00091F9F8E7A421002040420F00D82100203E
:100AC000DD37002070B50D4614461E4602F0AEF824
:100AD00050B9022E10D1012C0ED112A3D3E900235C
:100AE000C5E90023012007E0282C10D005D8012CEF
:100AF00009D0052C0FD0002070BD302CFBD10BA3EA
:100B0000D3E90023ECE70BA3D3E90023E8E70BA329
:100B1000D3E90023E4E70BA3D3E90023E0E700BF18
:100B2000AFF30080401DA12026812A0B78F6339F69
:100B300093CACD8D9E6AC421818A46EE2641727287
:100B4000DF25D7B7F017304A39059E5638B5054628
:100B50000E4C0021013500F0B7FBA4F82C55B4F879
:100B60002C0500F099FB78B1B4F82C0500F0A4FB3B
:100B7000014648B9B4F82C0500F0A6FBB4F82C35B2
:100B80000133A4F82C35EAE738BD00BFA8320020B5
:100B900010B50A4B0A4A1A6003F5805393F8602097
:100BA0003AB9DC6D2CB1204600F082FE204603F0FD
:100BB00053FEBDE81040034800F07ABED821002063
:100BC000404A0008203200202DE9F04F8FB000AFDE
:100BD00005460C4602F02AF8002849D1237E022B54
:100BE0001BD1E38A012B18D101F0FCFC0646FFF76C
:100BF000E1FD03464FF4C870DFF8C482B3FBF0F2A6
:100C000006F5167602FB103316FA83F3C8F80030A7
:100C1000E37E33B9A34B00221A703C37BD46BDE8D2
:100C2000F08F07F12401204600F0A2FC0028F4D147
:100C300007F11400FFF7D6FD97F8264007F11401DD
:100C4000224607F1270003F051FE0028E2D10F2CC5
:100C500008D8944B1C70D8F80030A3F51673C8F868
:100C60000030DAE797F82410284601F0D7FFD4E7E0
:100C7000E38A282B2BD010D8012B23D0052BCCD1E5
:100C8000BFF34F8F8849894BCA6802F4E06213436F
:100C9000CB60BFF34F8F00BFFDE7302BBDD1844E3B
:100CA000E17E327A9142B8D1607E3146002291F8DD
:100CB000DC50854200F0A5800132042A01F58A71DA
:100CC000F5D1AAE721462846FFF79CFDA5E7214676
:100CD0002846FFF703FEA0E7B2F8EC507B6005F171
:100CE00003094FEA99094FEA8902D11DC908A8EB07
:100CF000C1039D46EB460021584600F01FFB04F15E
:100D0000EE012A463144584600F006FB7B6813B9D1
:100D1000012000F0B7FA96F8D20000F0BDFA0446C0
:100D200030B9307200F0D8FA204600F0ABFAB1E0EA
:100D3000D6F8D4203AB996F8D200B6F82C258242DB
:100D400001D8FFF703FFD6F8D4202A44944208D2F2
:100D500096F8D200B6F82C250130824201D8FFF770
:100D6000F5FE70685FFA89F2594600F0EFFA08B9AB
:100D7000C54679E0726896F8D2002A447260D6F8C7
:100D8000D42005EB0209C6F8D49000F085FA81451D
:100D900009D396F8D220D6F8D4000132001B86F889
:100DA000D220C6F8D400FF2D0FD80024347200F0F2
:100DB00093FA204600F066FA00F000FD3D4B1881E2
:100DC00008B9FFF7A5FCC54627E7BB6896F8D90028
:100DD0000AFB0362FB68D2F8E41082F8E83001F500
:100DE0008061C2F8E030C2F8E410FFF7D5FDFFF7EC
:100DF00023FE96F8D920013202F0030286F8D920AA
:100E0000B6E74FF48A7A0AFB02F505F1EA013144AC
:100E1000204600F083FCF86000287FF4FEAE3544E5
:100E2000012285F8E82001F0DDFBD5F8E020D6EDC1
:100E3000007ADFED216A801A192838BF192040F6A0
:100E4000B832904228BF1046B8EE677A07EE900A93
:100E5000F8EEE77A67EEA67ADFED186AE7EE267A13
:100E6000FCEEE77AC6ED007A96F8D930BB60BA6836
:100E700073680AFB02F4321992F8E81059B1D2F8FB
:100E8000E4108B42E8463FF427AF002182F8E810D7
:100E9000C2F8E010C5467368064A9B0A0133138105
:100EA000BBE600BF9D21002000ED00E00400FA0534
:100EB000A83200208C110020CDCCCC3D6666663F68
:100EC000A0210020014B1870704700BF981100202E
:100ED00038B54FF00054134B22689A4220D1124B80
:100EE000627D12481A70237D03724FF48073C0F83C
:100EF000F8314FF40073C0F80C3300254FF4407301
:100F0000C0F820340A49C0F8E450C922093000F082
:100F100003FAE0222946204600F010FA012038BDED
:100F20000020FCE79AAD44C598110020A8320020AB
:100F30001600002037B500F041FC194D19492881F1
:100F40000223012218486B7101F0EAF90023019392
:100F5000164B174900931748174B4FF4805201F076
:100F600035FE164B197811B1124801F057FE01F009
:100F700039FB0446FFF71EFC4FF4C873B0FBF3F2D5
:100F800002FB130304F5167010FA83F00C4B186083
:100F900002F010FF08B10F232B8103B030BD00BF5A
:100FA0008C11002040420F00D8210020C50A000803
:100FB0009C110020A4210020C90B000898110020DA
:100FC000A02100202DE9F04F2DED028B8EA7D7E94F
:100FD00000670FF23C29D9E90089864C95B00DAD28
:100FE0009FED828BFFF728FDDFF82CB200230C93D6
:100FF000ADF83C300D936B6000230DF125028DEDB3
:10100000008B4FF0010A09A958468DF825308DF85C
:1010100024A001F035F99DF824200023002A40F097
:10102000AB80204601F002FE0546002847D1DFF8DC
:10103000ECB101F0D7FADBF8003098423FD301F071
:10104000D1FA0790FFF7B6FB079A4FF4C873B0FBCD
:10105000F3F101FB130302F5167010FA83F0CBF8DD
:101060000000DFF8BCB19BF800100791002914BF05
:101070002B46534610A88DF83030FFF7B3FB079985
:10108000C1F11002D2B2062A10AB28BF06221944C1
:101090000DF13100079200F03FF9079A0CAB039372
:1010A000182302930132544BD2B2CDE900A304922B
:1010B0003B463246204601F0FFFD8BF8005001F020
:1010C00091FA4E4A4E4D1368C31AB3F57A7F32D364
:1010D000106001F089FA02460B46204601F084FEBA
:1010E000204601F0A3FD30B32B7ADFF838A1002BA6
:1010F00014BF032302238AF8053001F073FA0DF1BF
:10110000400B4FF47A730122B0FBF3F05946CAF852
:101110000000504600F004FA18230293394B019363
:1011200080B240F25513CDE903B0009342464B46DE
:10113000204601F0C1FD2B7ACBB101F053FA4FF0FC
:10114000000A83464FF48A7295F8D900504400F0A3
:10115000030002FB005393F8E81089B30AF1010A77
:10116000BAF1040FF0D12B7A002B7FF438AF15B011
:10117000BDEC028BBDE8F08F4FF0904110A84A699A
:1011800082F010024A611946102200F0D7F80DF1E2
:1011900026030AAA0CA9584600F0F0FD95E80300C2
:1011A00011AB83E803009DF83C308DF84C300C9B6C
:1011B000109310A9DDE90A23204601F0E9FF1BE79F
:1011C000D3F8E01049B12B68FA2B38BFFA23ABEB08
:1011D00001010533B1EB430FC0D3FFF7DDFB4FF443
:1011E0008A720028BAD1BEE7AFF300800000000089
:1011F00000000000A42100209C210020D8370020FE
:10120000A8320020DC370020401DA12026812A0BB7
:10121000F1C6A7C1D068080FD8210020A021002066
:101220009D2100208C11002008B5054800F040FEEB
:10123000BDE80840034A0449002003F007BB00BF93
:10124000D821002018380020910B000870470000BA
:1012500070B502F013FC094E094D30800024286857
:101260003388834208D902F005FC2B68044401331B
:10127000B4F5D04F2B60F2D370BD00BF0C38002006
:10128000E037002002F086BC00F10060920000F51B
:10129000D04002F02DBC0000054B1A68054B1B889E
:1012A0009B1A834202D9104402F0E4BB002070472D
:1012B000E03700200C380020024B1B68184402F075
:1012C000DFBB00BFE0370020024B1B68184402F070
:1012D000E9BB00BFE0370020064991F8243033B164
:1012E0000023086A81F824300822FFF7CDBF0120CF
:1012F000704700BFE4370020022802BF4FF0904340
:1013000010229A6170470000022802BF4FF09043FC
:101310004FF480129A61704710B50023934203D0B6
:10132000CC5CC4540133F9E710BD0000034602460B
:10133000D01A12F9011B0029FAD170470244034662
:10134000934202D003F8011BFAE770472DE9F843F6
:101350001F4D144695F824200746884652BBDFF8F7
:1013600070909CB395F824302BB92022FF21484679
:101370002F62FFF7E3FF95F82400C0F10802A242B4
:1013800028BF2246D6B24146920005EB8000FFF707
:10139000C3FF95F82430A41B1E44F6B2082E174450
:1013A0009044E4B285F82460DBD1FFF795FF002874
:1013B000D7D108E02B6A03EB82038342CFD0FFF73B
:1013C0008BFF0028CBD10020BDE8F8830120FBE78C
:1013D000E43700202DE9F0470D46044600219046F1
:1013E000284640F27912FFF7A9FF23462022002168
:1013F000284601F06FFE231D02222021284601F01D
:1014000069FE631D03222221284601F063FEA31D0D
:1014100003222521284601F05DFE04F10803102275
:101420002821284601F056FE04F110030822382135
:10143000284601F04FFE04F11103082240212846FE
:1014400001F048FE04F1120308224821284601F069
:1014500041FE04F1140320225021284601F03AFEF7
:1014600004F1180340227021284601F033FE04F1F4
:1014700020030822B021284601F02CFE04F12103AC
:101480000822B821284601F025FE04F12207C026D3
:101490003B46314608222846083601F01BFEB6F5C9
:1014A000A07F07F10107F3D104F13203082231468E
:1014B000284601F00FFE002704F1330A94F8323079
:1014C0004FEAC7099F4209F5A47615D3B8F1000F7A
:1014D00008D1314604F599730722284601F0FAFD38
:1014E00009F24F16274694F832213B1B93420CD346
:1014F000F01DC008BDE8F0870AEB0703082231465B
:10150000284601F0E7FD0137D8E707F233133146EB
:101510000822284601F0DEFD08360137E3E7000027
:1015200013B504460846002101602346C0F80310A5
:101530002022019001F0CEFD0198231D02222021DE
:1015400001F0C8FD0198631D0322222101F0C2FDB4
:101550000198A31D0322252101F0BCFD019804F18F
:1015600008031022282101F0B5FD072002B010BDAC
:10157000F7B50023047F00910E4607221946054661
:1015800001F06CFC731C0093012200230721284604
:1015900001F064FCC4B9B31C009305222346082162
:1015A000284601F05BFC0D243746B278BB1B934202
:1015B00011D32B7FA88A0734E408BBB9844294BFB7
:1015C0000020012003B0F0BDAB8ADB00083BDB0844
:1015D000B3700824E8E7FB1C00932146002308228F
:1015E000284601F03BFC08340137DEE7201A18BF1B
:1015F0000120E7E7F7B50023047F00910E4608229B
:101600001946054601F02AFC731CC4B90822009350
:1016100011462346284601F021FC1024012372784C
:101620005F1C013B934211D32B7FA88A0734E40847
:10163000BBB9844294BF0020012003B0F0BDAB8A47
:10164000DB00083BDB0873700824E7E7F31900931D
:10165000214600230822284601F000FC08343B46BE
:10166000DDE7201A18BF0120E7E70000F8B50E46B5
:1016700005461446002181223046FFF75FFE2B46C7
:1016800008220021304601F025FD7CB96B1C0722A1
:101690000821304601F01EFD0F2401236A785F1CEB
:1016A000013B934204D3E01DC008F8BD0824F4E7D1
:1016B000EB1921460822304601F00CFD08343B4668
:1016C000ECE70000F8B50E46054614460021CE2290
:1016D0003046FFF733FE2B4628220021304601F02A
:1016E000F9FC7CB905F1080308222821304601F0F5
:1016F000F1FC30242F462A7A7B1B934204D3E01D51
:10170000C008F8BD2824F5E707F10903214608229F
:10171000304601F0DFFC08340137ECE7F7B5047F11
:1017200000910E46012310220021054601F096FB90
:10173000C4B9B31C0093092223461021284601F0A6
:101740008DFB192437467288BB1B9A4211D82B7F18
:10175000A88A0734E408BBB9844294BF0020012062
:1017600003B0F0BDAB8ADB00103BDB0873801024B4
:10177000E8E73B1D0093214600230822284601F09C
:101780006DFB08340137DEE7201A18BF0120E7E7B8
:1017900030B5094D0A4491420DD011F8013B584033
:1017A000082340F30004013B2C4013F0FF0384EABC
:1017B0005000F6D1EFE730BD2083B8EDF7B5364ADB
:1017C000106851686B4603C36A463449344808239D
:1017D00003F09CF8044690BB0A25324A1068516811
:1017E0006B4603C36A4630492D48082303F08EF840
:1017F0000446002847D00369B3F5663F43D8B0F8E4
:101800006620B2F57B7F3ED1284A024402F15C019A
:101810008B4238D35C3B224900209E1AFFF7B8FF69
:101820003246074604F164010020FFF7B1FFA368C8
:101830009F4228D1E368984208BF002523E003694E
:10184000B3F5663F26D8428BB2F57B7F20D1174A8D
:10185000024402F110018B4218D3103B10490020C2
:101860009D1AFFF795FF2A46064604F1180100204D
:10187000FFF78EFFA3689E4202D1E368984201D031
:101880000D25AAE70025284603B0F0BD1025A4E7E2
:101890000C25A2E70B25A0E7044A0008DC9703000B
:1018A000006800080D4A0008909703000898FFF7A9
:1018B00010B5037C044613B9006803F00FF8204606
:1018C00010BD00000023BFF35B8FC360BFF35B8FCD
:1018D000BFF35B8F8360BFF35B8F7047BFF35B8F9A
:1018E0000068BFF35B8F704770B505460C30FFF79B
:1018F000F5FF05F1080604463046FFF7EFFFA0426A
:1019000006D930466D68FFF7E9FF2544281A70BDF7
:101910003046FFF7E3FF201AF9E7000070B50546EF
:10192000406898B105F10800FFF7D8FF05F10C06F3
:1019300004463046FFF7D2FF8442304694BF6D68BC
:101940000025FFF7CBFF013C2C44201A70BD00009E
:1019500038B50C460546FFF7C7FFA04210D305F186
:101960000800FFF7BBFF04446868B4FBF0F100FB1C
:101970001144BFF35B8F0120AC60BFF35B8F38BDB8
:101980000020FCE72DE9F041144607460D46FFF71D
:10199000C5FF844228BF0446D4B1B84658F80C6B42
:1019A0004046FFF79BFF3044286040467E68FFF7C3
:1019B00095FF331A9C4203D86C600120BDE8F0818A
:1019C0006B60A41B3B68AB602044E8600220F5E735
:1019D0002046F3E738B50C460546FFF79FFFA042C7
:1019E00010D305F10C00FFF779FF04446868B4FBDD
:1019F000F0F100FB1144BFF35B8F0120EC60BFF3FB
:101A00005B8F38BD0020FCE72DE9FF418846694621
:101A10000746FFF7B7FF6C4606B204EBC606002583
:101A2000B44209D06268206808EB0501FFF774FC36
:101A3000636808341D44F3E729463846FFF7CAFFB8
:101A4000284604B0BDE8F081F8B505460C300F46D5
:101A5000FFF744FF05F1080604463046FFF73EFF56
:101A6000A042304688BF6C68FFF738FF201A386004
:101A700020B130462C68FFF731FF2044F8BD00004C
:101A800073B5144606460D46FFF72EFF844228BF65
:101A900004460190DCB101A93046FFF7D5FF019B58
:101AA00033B93268C5E90233C5E9002401200CE0EE
:101AB0009C4238BF01942860019868608442F5D93F
:101AC0003368AB60241AEC60022002B070BD20467F
:101AD000FBE700002DE9FF410F466946FFF7D0FF05
:101AE0006C4600B204EBC0050026AC4209D0D4F825
:101AF000048054F8081BB8194246FFF70DFC464411
:101B0000F3E7304604B0BDE8F081000038B5054683
:101B1000FFF7E0FF044601462846FFF719FF20467D
:101B200038BD0000302383F3118862B6704700008F
:101B3000002383F3118862B67047000010B4026876
:101B400054681A4623465DF8044B18470120704735
:101B50000020704700207047704700000020704749
:101B60000E20704700F5805090F8C800C0F3400088
:101B70007047000000F5805090F9C90070470000E0
:101B8000F7B50C68BDF8207014F000541E466FD1F4
:101B90000B7B082B6CD8FFF7C5FF4569AB685B0171
:101BA0000CD4AB681B0108D4AC6814F080545DD130
:101BB000FFF7BEFF204603B0F0BD01240B6804F11F
:101BC000180C002BB8BFDB004FEA0C1CB4BF43F06D
:101BD00004035B0545F80C300B680FFA84FC13F026
:101BE000804F18BF05EB0C1E05EB0C1C1EBFDEF86A
:101BF000803143F00203CEF880310B7BCCF8843186
:101C000005EB04158B68C5F88C314B68C5F8883135
:101C1000DCF8803143F00103CCF8803100EB44154F
:101C200041F268031D4403EB44130344C5E9002655
:101C300008330D4601F10C0C55F804EB43F804EBA6
:101C40006545F9D184342D881D8000EB441407F0DC
:101C50000303257925F00B052B432371FFF768FF5C
:101C60000097334600F0E0FC0120A4E70224A5E73A
:101C70004FF0FF309FE7000013B500F5805401914D
:101C8000E06DFFF74BFE1F280AD90199E06D202275
:101C9000FFF7BAFEA0F120035842584102B010BD30
:101CA0000020FBE708B500F58050FFF73BFFC06D53
:101CB000FFF708FEBDE80840FFF73ABF00220260C8
:101CC000828142608260704710B500220023C0E923
:101CD00000230023044603810C30FFF7EFFF20466A
:101CE00010BD0000F0B5054600F580500C4690F898
:101CF000C83013F0040FC3F3800108BF114661F32D
:101D0000820304F1840680F8C83005EB461389B0DD
:101D10001B79D8072ED57AB319072DD46846FFF75B
:101D2000D3FF05EB441303F5835303F1180703AA0C
:101D3000103318685968144603C40833BB4222465E
:101D4000F7D1186820609B88A380DDE90E23CDE9D8
:101D500000230123ADF808302B686946DB6B284669
:101D6000984705EB46152B791A075CBF43F008032B
:101D70002B7101E0002AF4D109B0F0BD2DE9F04744
:101D8000074688B007F5805468469A468846FFF7AC
:101D9000C9FE9146FFF798FFE06DFFF7A5FD1F28EC
:101DA00029D9E06D20226946FFF7B0FE202822D114
:101DB00003AD444605AB2E4603CE9E4220606160D3
:101DC000354604F10804F6D130682060B388A3805A
:101DD000DDE90023C9E90023BDF80830AAF8003086
:101DE000FFF7A6FE4A4653464146384608B0BDE8CE
:101DF000F04700F007BCFFF79BFE002008B0BDE8ED
:101E0000F08700002DE9F84F0023C0E90133254B8E
:101E1000044640F8183B0F46FFF750FF04F1280036
:101E2000FFF752FF04F1480804F58255464608358D
:101E300030462036FFF748FFAE42F9D104F5805511
:101E40004FF480534FF00009C5E91339C5F84880B5
:101E50000123EE6504F5875804F58456C5F85490BF
:101E600085F8583085F86030083608F108084FF0DA
:101E7000000A4FF0000B46E908ABA6F11800FFF787
:101E80001DFF203646F8289C4645F4D185F8C970D8
:101E900017B1054800F0A0FB044B63612046BDE884
:101EA000F88F00BF404A0008184A0008006400404C
:101EB00010B5044B197804464A1C1A70FFF7A2FFAC
:101EC000204610BD143800202DE9F047002950D0DD
:101ED000294B2A4FB7FBF1F599428CBF0A231123F6
:101EE000581EB5FBF3FC03FB1C53C4B22BB10228F4
:101EF0000346F5D80020BDE8F0870CF1FF36B6F5B3
:101F0000806FF7D2C4EBC40E0EF103034FEAE3096E
:101F1000C3F3C703A4EB030809F1010A4FF47A7570
:101F20005FFA88F009FB05555AFA88F8B5FBF8F511
:101F3000B5F5617FC1BF0EF1FF33C3F3C703E01AEC
:101F4000C0B25C1C50FA84F40CFB04F4B7FBF4F44C
:101F5000A142CFD1013BDBB20F2BCBD80138C0B2AD
:101F60000728C7D80021107116809170D370012006
:101F7000C1E70846BFE700BF3F420F0000512502FE
:101F800070B505460E464FF47A746B695B6803F0D2
:101F90000103B3424FF0010004D001F0A5FC013C65
:101FA000F3D1204670BD000030B54269936913F04B
:101FB000700F16D000230B4C936103F1840200EBE9
:101FC000421211794D0709D5890707D5416954F89F
:101FD00023508D60117941F0040111710133032BFD
:101FE000EBD130BD2C4A000873B51D464369164637
:101FF0009A68D207044609D59A6801219960C2F30C
:102000004002CDE900650021FFF76CFE63699A6824
:10201000D1050BD59A684FF480719960C2F34022C4
:10202000CDE9006501212046FFF75CFE63699A68EF
:10203000D2030BD59A684FF480319960C2F34042C5
:10204000CDE9006502212046FFF74CFE204602B094
:10205000BDE87040FFF7A8BFF8B5044646690029FF
:102060006CD106F10C07386880076AD006EB0115C1
:102070003868D5F8B00110F0040FD5F8B0011ABFD8
:10208000C00840F00040400DA061D5F8B0C11CF080
:10209000020F1CBF40F08040A061D5F8B40106EBF0
:1020A000011100F00F0084F82400D1F8B801207766
:1020B000D1F8B801000A6077D1F8B801000CA07718
:1020C000D1F8B801000EE077D1F8BC0184F8200007
:1020D000D1F8BC01000A84F82100D1F8BC01000C41
:1020E00084F82200D1F8BC11090E84F8231038219D
:1020F000396004F1340004F1180104F1240551F8A9
:10210000046B40F8046BA942F9D109880180C4E945
:102110000A2321460023238651F8283B2046DB6B07
:10212000984704F58052204692F8C83043F00403E3
:1021300082F8C830BDE8F840FFF736BF06F1100757
:1021400091E7F8BD10B5044600F04EFA02460B4682
:1021500052EA030102D0013A63F10003044908681E
:1021600020B12146BDE81040FFF776BF10BD00BF8B
:1021700010380020F8B500F583511E46FFF7D2FC59
:10218000DFF844C00831002404F1840500EB451554
:102190002B795F070ED4DB060CD5D1E9007397428B
:1021A000B34107D243695CF824709F602B7943F0F8
:1021B00004032B710134032C01F12001E4D1BDE8AB
:1021C000F840FFF7B5BC00BF2C4A000808B5FFF780
:1021D000A9FCFFF7E9FEBDE80840FFF7A9BC000035
:1021E000F8B543690546986800F0E050B0F1E05F4B
:1021F0000F461FD0E8B1FFF795FC05F58354103466
:10220000002606F1840305EB43131B791A0706D554
:102210000136032E04F12004F3D1012007E05B070F
:10222000F6D42146384600F039FA0028F0D1FFF7FD
:102230007FFCF8BD0120FCE700F5805008B5FFF7F2
:1022400071FCC06DFFF750FBFFF772FC43090CBF38
:102250000120002008BD0000F8B51D4600231370C2
:102260000F4606461446FFF7E7FF80F0010038707E
:1022700025B129463046FFF7B3FF2070F8BD0000B6
:102280002DE9B8410C4615461F46804600F0ACF9D2
:102290000B462178024609B9287850B14046FFF72D
:1022A00069FFFFF793FF3B462A462146FFF7D4FF1D
:1022B0000120BDE8B881000010B5FFF733FC174BD3
:1022C000DA6942F00072DA611A6942F000721A614A
:1022D0001A6900F5805422F000721A61FFF728FC99
:1022E00094F8C830DB0718D4B9B103211320FFF7E5
:1022F00019FC01F0C7F90321142001F0C3F90321EF
:10230000152001F0BFF994F8C83043F0010384F8B8
:10231000C830BDE81040FFF70BBC10BD00100240F4
:102320002DE9F04700F5805588B095F8C930012BAC
:102330000446884616467FD8804F57F823200AB9AE
:1023400047F82300D7F800A0C4F80C802674BAF12F
:10235000000F63D095F8C930012B6FD001212046C2
:10236000FFF7AAFFFFF7DEFB6269136823F00203A1
:1023700013606269136843F0010313606369002707
:102380005F6101212046FFF7D3FBFFF7F9FD00282D
:1023900000F09580E86DFFF795FA04F58359BA4689
:1023A00009F10809202200216846FEF7C7FF02A8AC
:1023B000FFF784FCCDF818A06A4609EB07030DF17E
:1023C000180E9446BCE80300F44518605960624654
:1023D00003F10803F5D1DCF80000186020379CF801
:1023E00004201A71602FDDD195F8C8306FF3820395
:1023F000002785F8C8306A4641462046ADF800708F
:10240000ADF802708DF80470FFF75EFD636948BB9C
:102410004FF400421A6008B0BDE8F08741F2D000E6
:1024200002F01CFA814610B15146FFF7EBFCC7F8E9
:102430000090B9F1000F8DD10020ECE738680368F7
:102440001B6B98470146002888D13868FFF734FF96
:102450003868036832465B684146984700287FF435
:102460007DAFE9E761221A609DF802309DF80320F4
:102470001B06120402F4702203F040731343BDF8EC
:102480000020C2F3090213439DF804201205022E16
:1024900002F4E0020CBF4FF00041002113436269D7
:1024A0000B43D361636913225A616269136823F095
:1024B0000103136039462046FFF762FD08B96369DE
:1024C000A6E795F8C93093BB6169D1F8002242F0C4
:1024D0000102C1F800226169D1F8002222F47C5285
:1024E00022F00E02C1F800226169D1F8002242F404
:1024F0006062C1F800226269C2F814326269C2F8EF
:102500000432626941F6FF71C2F80C126269C2F8C6
:1025100040326269C2F8443263690122C3F81C2266
:102520006269D2F8003223F00103C2F8003295F854
:10253000C83043F0020385F8C8306CE7103800203B
:1025400008B500F051F850EA0103024602D0421EDD
:1025500061F10001044B186810B10B46FFF744FD10
:10256000BDE8084001F064B81038002008B500202C
:10257000FFF7E8FDBDE8084001F05AB808B50120B2
:10258000FFF7E0FDBDE8084001F052B800B59BB090
:10259000EFF3098168226846FEF7BEFEEFF305837C
:1025A000014B9B6BFEE700BF00ED00E008B5FFF7B5
:1025B000EDFF000000B59BB0EFF30981682268468B
:1025C000FEF7AAFEEFF30583014B5B6BFEE700BF4E
:1025D00000ED00E0FEE700000FB408B5029801F03E
:1025E00019F9FEE701F02EBB01F004BB13B56C46F0
:1025F00084E80600031D94E8030083E80500012039
:1026000002B010BD73B58568019155B11B885B0799
:1026100007D4D0E900369B6B9847019AC1B2304687
:10262000A847012002B070BDF0B5866889B00546A4
:102630000C465EB1BDF838305B070AD4D0E90037EC
:102640009B6B98472246C1B23846B047012009B07B
:10265000F0BD00220023CDE900230023ADF80830AF
:102660000A4603AB01F10806106851681C4603C412
:102670000832B2422346F7D1106820609288A280C7
:10268000FFF7B2FF0423ADF808302B68CDE9000155
:10269000DB6B694628469847D8E7000030B50368E9
:1026A0000968DD0FB5EBD17F23F0604421F0604273
:1026B0004FEAD1700BD0002BB8BFA40C0029B8BFD3
:1026C000920C944202D034BF0120002030BD9442CD
:1026D00005D1C1F38070C3F380738342F6D1944275
:1026E0002CBF00200120F1E72DE9F041456A15B922
:1026F0004162BDE8F0814B6823F06047C3F38A462E
:102700004FEAD37EC3F3807816EA230638BF3E46ED
:10271000AC462B465A68BEEBD27F22F060440AD00A
:10272000002A18DAA40CB44217D19D420FD10D60D3
:10273000DEE71346EEE7A74207D102F08044C2F37A
:10274000807242450BD054B1EFE708D2EDE7CCF8E8
:1027500000100B60CDE7B44201D0B442E5D81A684E
:102760009C46002AE5D11960C3E700002DE9F04737
:10277000089D01F007044FEAD508224405F007053B
:1027800000EBD1004FF47F49944201D1BDE8F087BE
:1027900004F0070705F0070A57453E4638BF56467E
:1027A000C6F10806111B8E4228BF0E46E10808EB51
:1027B000D50E415C13F80EC0B94029FA06F721FA8C
:1027C0000AF1FFB28CEA010147FA0AF739408CEAB4
:1027D000010C03F80EC034443544D5E780EA0120EB
:1027E000082341F2210201B24000002980B203F126
:1027F000FF33B8BF504013F0FF03F4D1704700001F
:1028000038B50C468D18A54200D138BD14F8011B0F
:10281000FFF7E4FFF7E7000042684AB1136843603E
:102820004389818901339BB29942438138BF8381B7
:102830001046704770B588B0202204460D466846A1
:102840000021FEF77BFD20460495FFF7E5FF0246D9
:1028500058B16B46054608AE1C4603CCB44228600E
:102860006960234605F10805F6D1104608B070BD31
:10287000082817D909280CD00A280CD00B280CD00E
:102880000C280CD00D280CD00E2814BF402030206E
:1028900070470C2070471020704714207047182094
:1028A0007047202070470000082817D90C280CD941
:1028B00010280CD914280CD918280CD920280CD988
:1028C00030288CBF0F200E207047092070470A2047
:1028D00070470B2070470C2070470D207047000098
:1028E0002DE9F843078C072F04461ED9D0E902983A
:1028F00000254FF6FF73C5F12006A5F1200029FA47
:1029000005F108FA06F628FA00F031430143C9B28E
:102910001846FFF763FF0835402D0346EBD1E16908
:102920003A46BDE8F843FFF76BBF4FF6FF70BDE8CE
:10293000F883000010B54B6823B9CA8A63F3090213
:10294000CA8210BD04691A681C600361C38A013B16
:10295000C3824A60EFE700002DE9F84F1D46CB8A9D
:102960000F46C3F309010529814692460B4630D034
:102970000020AAB207F11A049EB2042E1FFA80F8B2
:102980000FD8904503F1010306D3FB8A0A4462F392
:102990000903FB8201201AE01AF80060E6540130B6
:1029A000EAE79045F1D2A1F1050B1C237C68BBFB43
:1029B000F3F203FB12BB1FFA8BF6002C45D14846FD
:1029C000FFF72AFF044638B978606FF00200BDE8CF
:1029D000F88F4FF00008E6E7002606607860ADB299
:1029E0004FF0000B454510D90AEB0803221D13F8E0
:1029F000011B9155B1B208F101081B291FFA88F893
:102A00002BD0454506F10106F1D8FB8AC3F3090234
:102A1000154465F30903BCE7013292B21C462368F2
:102A2000002BF9D16B1F0B441C21B3FBF1F30133D5
:102A30009BB29A42D3D2BBF1000FD0D14846FFF7E8
:102A4000EBFE20B9C4F800B0BFE70122E7E7C0F809
:102A500000B05E4620600446C1E74545D5D94846EA
:102A6000FFF7DAFE08B92060AFE7C0F800B0002633
:102A700020600446B6E700002DE9F04F2DED028BF3
:102A80001C4683B05B69019207468846002B00F024
:102A90009A80238C2BB1E269002A00F09480072BE6
:102AA00035D807F10C00FFF7B7FE054638B96FF0CF
:102AB0000205284603B0BDEC028BBDE8F08F14225E
:102AC0000021FEF73BFC228CE16905F10800FEF7CE
:102AD00023FC208C013080B2FFF7E6FEFFF7C8FE32
:102AE000013880B22084013028746369228C1B78FD
:102AF0002A4403F01F0363F03F0348F000411372C0
:102B0000384669602946FFF7EFFD0125D1E700F15E
:102B10000C034FF0000908EE103A4FF0800A4E46C1
:102B20004D4618EE100AFFF777FE83460028BED008
:102B300014220021FEF702FC002E3AD1019BABF8D3
:102B4000083002220BF1080E1FFA82FC0CF1010082
:102B5000BCF1060F218C80B201D88E422BD3FFF737
:102B6000A3FEFFF785FE62691278013802F01F02AA
:102B70008E4208BF4FF0400A42EA49121BFA80F128
:102B80004AEA020A013048F0004281F808A08BF8B6
:102B90001000CBF8042059463846FFF7A5FD238CDA
:102BA0000135B3422DB289F001094FF0000AB8D1C6
:102BB0007FE70022C6E7E169895D0EF80210013661
:102BC000B6B20132C0E76FF0010572E7F8B51546FD
:102BD0000E463022002104461F46FEF7AFFB069B3F
:102BE0006360B5F5001F079BA76034BF6A094FF605
:102BF000FF72A36297B2E66104F1100000239A42CB
:102C000006D800230360A782E3822383E360F8BD34
:102C10000660013330462036F1E7000003781BB927
:102C20004BB2002BC8BF017070470000007870479E
:102C3000F8B50C46C969074611B9238C002B37D16A
:102C4000257E1F2D34D8387828BB228C072A2CD813
:102C5000268A36F003032BD14FF6FF70FFF7D0FD25
:102C600020F001003102400441EA0561400C41EAD4
:102C700040254FF6FF72234629463846FFF7FCFEF3
:102C8000002807DD626913780133DBB21F2B88BF90
:102C900000231370F8BD218A2D0645EA012505435E
:102CA0002046FFF71DFE0246E5E76FF00300F1E75F
:102CB0006FF00100EEE7000070B58AB004461646DA
:102CC0000021282268461D46FEF738FBBDF8383043
:102CD000ADF810300F9B05939DF840308DF81830FB
:102CE000119B07936946BDF84830ADF82030204667
:102CF000CDE90265FFF79CFF0AB070BD2DE9F041F8
:102D0000D36905460C4616460BB9138C5BBB377E60
:102D10001F2F28D895F80080B8F1000F26D0304634
:102D2000FFF7DEFD3378210241EAC33141EA0801B1
:102D3000338A41EA076141EA03410246334641F0E2
:102D400080012846FFF798FE00280ADD3378012B22
:102D500007D1726913780133DBB21F2B88BF0023C0
:102D60001370BDE8F0816FF00100FAE76FF0030027
:102D7000F7E70000F0B58BB004460D46174600217A
:102D8000282268461E46FEF7D9FA9DF84C305A1E96
:102D9000534253418DF800309DF84030ADF810306B
:102DA000119B05939DF848308DF81830149B0793BC
:102DB0006A46BDF85430ADF8203029462046CDE9AA
:102DC0000276FFF79BFF0BB0F0BD0000406A00B138
:102DD00004307047436A1A68426202691A600361EC
:102DE000C38A013BC38270472DE9F041D0F82080AF
:102DF000194E14461D464146002709B9BDE8F08129
:102E0000D1E90223A21A65EB0303964277EB030391
:102E10001ED2036A8B420DD1FFF78CFD036A1B683B
:102E2000036203690B60C38A0161016A013BC382CB
:102E30008846E2E7FFF77EFD0B68C8F800300369BB
:102E40000B60C38A0161013BC382D8F80010D4E74C
:102E500088460968D1E700BF80841E002DE9F04F45
:102E60008BB00D46DDF8509014469B4680460028F6
:102E700000F01981B9F1000F00F01581531E3F2BAE
:102E800000F21181012A03D1BBF1000F40F00B8148
:102E90000023CDE90833B8F81430B5EBC30F4FEA7F
:102EA000C30703D300200BB0BDE8F08F2B199F425E
:102EB000D8F80C303ABF7F1BFFB227461BB9D8F8B1
:102EC0001030002B7AD0272D4ED8C5F12806B742F6
:102ED0004FF000032CBFF6B23E4600932946D8F8C7
:102EE000080008AB3246FFF741FCA7EB060A354461
:102EF0005FFA8AFAB8F8143003F10053053BDB009F
:102F00000493D8F80C3003932821039B13B1BAF132
:102F1000000F2CD1D8F8100040B1BAF1000F05D045
:102F2000009608AB5246691AFFF720FC38B2002F12
:102F3000B8D066070AD00AAB03EBD401624211F89D
:102F4000083C02F00702134101F8083C082C3CD968
:102F5000102C40F2B580202C40F2B780BBF1000F5E
:102F600000F09C80082334E0BA460026C2E7049BA8
:102F7000E02B28BFE02306930B44AB42059314D902
:102F80005A1B03980096924534BF5246D2B2691A32
:102F900008AB04300792FFF7E9FB079A1644AAEB47
:102FA000020A1544F6B25FFA8AFA049B069A05995A
:102FB0009B1A0493039B1B680393A6E70093D8F81E
:102FC000080008AB3A462946AEE7BBF1000F13D024
:102FD0000123B4EBC30F6CD0082C12D89DF820301D
:102FE000621E23FA02F2D50706D54FF0FF3202FA2D
:102FF00004F423438DF820309DF8203089F8003008
:1030000051E7102C12D8BDF82030621E23FA02F2CC
:10301000D10706D54FF0FF3202FA04F42343ADF88E
:103020002030BDF82030A9F800303CE7202C0FD824
:103030000899631E21FA03F3DA0705D54FF0FF3232
:1030400002FA04F40C430894089BC9F800302AE7FC
:10305000402C2BD0DDE90865611EC4F12102A4F1EA
:10306000210326FA01F105FA02F225FA03F31143CE
:103070001943CB0712D50122A4F12003C4F120018A
:1030800002FA03F322FA01F1A240524243EA010399
:1030900063EB430332432B43CDE90823DDE90823E7
:1030A000C9E90023FFE66FF00100FCE66FF00800BD
:1030B000F9E6082CA0D9102CB3D9202CEED8C3E700
:1030C000BBF1000FADD0022383E7BBF1000FBBD0F3
:1030D00004237EE730B5012A144638BF0124402C72
:1030E00085B028BF40240025012ACDE9025518D813
:1030F0001B788DF8083063070AD004AB03EBD405C6
:10310000624215F8083C02F00702934005F8083CBB
:10311000009103462246002102A8FFF727FB05B0D5
:1031200030BD082AE4D9102A03D81B88ADF808302E
:10313000E1E7202A8DBFD3E900231B680293CDE984
:103140000223D8E710B5CB681BB98B600B618B826B
:1031500010BD04691A681C600361C38A013BC38205
:10316000CA60F0E703064CBFC0F3C03002207047CE
:1031700008B50246FFF7F6FF022806D15306C2F350
:103180000F2001D100F0030008BDC2F30740FBE7A8
:103190002DE9F04F93B0CDE903230A6804461046A9
:1031A000FFF7E0FF022814BFC2F306260026002A1C
:1031B0000D46824680F2F28112F0C04940F0EE8165
:1031C000097B002900F0EA81022803D02378B3426A
:1031D00040F0E781C2F304630693104602F07F03D8
:1031E0000593FFF7C5FF059B29444FEA834848EA4A
:1031F0000A4848EA4668CE7800230022CDE9082331
:10320000F309834648EA0008029367D0059B0093C0
:1032100002466768534608A92046B847002800F0D0
:10322000C381276A4FB9414604F10C00FFF702FB46
:10323000074690B96FF0020054E03B6998450DD005
:103240003F68002FF9D1414604F10C00FFF7F2FA74
:1032500007460028EED0236A3B60276297F817C024
:1032600006F01F08CCF3840CACEB08001FFA80FEBC
:103270000028B8BF0EF12000A8EB0C031FFA83FE54
:10328000D7E90221B8BF00B2002B0793BEBF0EF1F1
:1032900020031BB2079352EA010338D0039BDFF8E7
:1032A00024E39A1A049B4FF0000C63EB010196454E
:1032B0007CEB01032BD36B7B97F81AE0734519D194
:1032C000029B002B78D0012821DC7868F8B9DFF860
:1032D000F0C2944570EB010316D337E0276A27B993
:1032E0006FF00C0013B0BDE8F08F3B699845B5D086
:1032F0003F68F4E7B24890427CEB010301D3002021
:10330000F0E7029B002BFAD0079B0F2B17DCFA7D0E
:10331000B30002F0030203F07C031343FB7539464C
:103320002046FFF707FB6B7BBB76029B3BB9FB7D1F
:10333000C3F38402013262F38603FB75D0E76A7B34
:10334000BB7E9A42DBD1029B002B35D0B309022B06
:1033500032D0039BBB60049BFB60142200210DA8AC
:10336000FDF7ECFF039B0A93049B0B932B1D0C931F
:103370002B7BADF83EB0013BDBB2ADF83C30069B99
:103380008DF84230059B8DF8433094F82C308DF841
:1033900040A083F001038DF844308DF84180A3688C
:1033A0000AA920469847FB7DC3F38403013303F049
:1033B0001F039B02FB82A2E7FB7DC6F34012B2EB28
:1033C000D31F40F0F480C3F38403434540F0F28000
:1033D000029A2B7BB609002A4DD0F2075DD4032B4D
:1033E00040F2EB80039BBB60049BFB602B7BAE1D1C
:1033F000033BDBB23246394604F10C00FFF7ACFA6E
:1034000000280CDA39462046FFF794FAFB7DC3F317
:103410008403013303F01F039B02FB820AE7DDE90B
:103420000884AB883B834FF6FF73C9F12000A9F1F4
:10343000200228FA09F104FA00F0014324FA02F20A
:1034400011431846C9B2FFF7C9F909F10809B9F1E2
:10345000400F0346E9D1B8822A7B033AD2B2314603
:10346000FFF7CEF9FB7DB882DA43C2F3C01262F3F4
:10347000C713FB7543E786B92E1D013BDBB232460D
:10348000394604F10C00FFF767FA0028BADB2A7B03
:10349000B88A013AD2B23146E2E7F98AC1F30901AA
:1034A000013B0429DAB25BD8281D002307F11B0673
:1034B0009A4208D910F801CB06F801C00131013356
:1034C0000529DBB2F4D103990A9104990B91934237
:1034D00007F11B010C9138BF043379680D9134BF9B
:1034E00055FA83F300230E93FB8AADF83EB0C3F385
:1034F00009031A44069B8DF84230059B8DF8433032
:1035000094F82C30ADF83C2083F001038DF8443062
:1035100000238DF840A08DF841807B602A7BB88A1B
:10352000013A291DFFF76CF93B8BB882834203D126
:10353000A3680AA92046984720460AA9FFF702FE79
:10354000FB7DBA8AC3F38403013303F01F039B029C
:10355000FB823B8B9A420CBF00206FF01000C1E64B
:103560007B68002BAFD0052001E01C3033461E687D
:10357000002EFAD1091A081D2E1D184401EB090C62
:10358000BCF11B0F5FFA89F39DD89A429BD916F8BC
:10359000013B00F8013B09F10109EFE76FF0090079
:1035A000A0E66FF00A009DE66FF00B009AE66FF060
:1035B0000D0097E66FF00E0094E66FF00F0091E6B5
:1035C00040420F0080841E00EFF3098305494A6BD7
:1035D00022F001024A63683383F30988002383F3EE
:1035E0001188704700EF00E0302080F3118862B648
:1035F0000C4B0D4AD96821F4E0610904090C0A4317
:10360000DA60D3F8FC20094942F08072C3F8FC204C
:103610000A6842F001020A602022DA7783F8220069
:10362000704700BF00ED00E00003FA05001000E065
:1036300010B5302383F311880E4B5B6813F40063DD
:1036400014D0F1EE103AEFF30984683C4FF0807328
:10365000E361094BDB6B236684F3098800F098F87B
:1036600010B1064BA36110BD054BFBE783F3118836
:10367000F9E700BF00ED00E000EF00E003060008FE
:103680000606000800F1604303F561430901C9B271
:1036900083F80013012200F01F039A4043099B00A6
:1036A00003F1604303F56143C3F880211A6070475A
:1036B00000F16040090100F56D40C9B20176704724
:1036C00000230375826803691B6899689142FBD2E5
:1036D0005A680360426010605860704700230375A9
:1036E000826803691B6899689142FBD85A68036035
:1036F000426010605860704708B50846302383F375
:1037000011880B7D032B05D0042B0DD02BB983F32F
:10371000118808BD8B6900221A604FF0FF33836166
:10372000FFF7CEFF0023F2E7D1E9003213605A60C1
:10373000F3E70000FFF7C4BF054BD96808751868A8
:1037400002681A60536001220275D860FCF744BF1A
:103750002038002030B50C4BDD684B1C87B0044688
:103760000FD02B46094A684600F0FEF82046FFF7C6
:10377000E3FF009B13B1684600F000F9A86907B0A9
:1037800030BDFFF7D9FFF9E720380020F9360008EF
:10379000044B1A68DB6890689B68984294BF0020CD
:1037A0000120704720380020084B10B51C68D868ED
:1037B00022681A60536001222275DC60FFF78EFFD9
:1037C00001462046BDE81040FCF706BF2038002027
:1037D000044B1A68DB6892689B689A4201D9FFF72C
:1037E000E3BF70472038002038B5074C0749084828
:1037F000012300252370656000F00AFB022323707B
:1038000085F3118838BD00BF483A0020844A00087B
:103810002038002008B572B6044B186500F0CEF9C8
:1038200000F092FA024B03221A70FEE720380020C3
:10383000483A002000F0B4B8EFF3118020B9EFF35C
:103840000583302282F311887047000010B530B92B
:10385000EFF30584C4F3080414B180F3118810BD9C
:10386000FFF7B6FF84F31188F9E700008B600223AD
:1038700008618B82084670478368A3F1840243F88D
:10388000142C026943F8442C426943F8402C094A3D
:1038900043F8242CC26843F8182C022203F80C2C9D
:1038A000002203F80B2C044A43F8102CA3F120004B
:1038B000704700BFF10500082038002008B5FFF769
:1038C000DBFFBDE80840FFF735BF0000024BDB68B7
:1038D00098610F20FFF730BF20380020302383F39A
:1038E0001188FFF7F3BF000008B50146302383F3CA
:1038F00011880820FFF72EFF002383F3118808BDED
:10390000064BDB6839B1426818605A601360436047
:103910000420FFF71FBF4FF0FF3070472038002012
:103920000368984206D01A68026050609961184690
:10393000FFF700BF7047000010B50A4C23699A6872
:1039400091420CD85A6881600360426010609A68A6
:103950005860511A99604FF0FF33A36110BD1B6886
:10396000891AECE72038002010B4C0E903230023B3
:103970005DF8044B4361FFF7DFBF00000368816817
:103980009A680A449A60426813605A600023036090
:10399000024B4FF0FF329A61704700BF2038002081
:1039A00070B5124DEB692A460133EB6152F8103FB6
:1039B000934206D09A68013A9A6030262C69A3682F
:1039C00003B170BDD4E900210A605160236083F324
:1039D0001188D4E903312046984786F3118861693C
:1039E0000029EBD02046FFF7A7FFE7E720380020AB
:1039F00000207047FEE70000704700004FF0FF30E6
:103A000070470000BFF34F8F024AD368DB07FCD436
:103A1000704700BF0020024008B5074B1B7853B920
:103A2000FFF7F0FF054B1A69120641BF044A5A60BE
:103A300002F188325A6008BD603A0020002002403E
:103A40002301674508B5054B1B7833B9FFF7DAFF4B
:103A5000034A136943F08003136108BD603A0020F4
:103A6000002002407F289ABF00F58030C00200206D
:103A7000704700004FF400607047000080207047DE
:103A80007F2808B50BD8FFF7EDFF00F5006302684B
:103A9000013204D104308342F9D1012008BD002055
:103AA000FCE700007F2810B504461CD8FFF7AAFFEA
:103AB000FFF7B2FF0D4BF322DA6002221A61FFF723
:103AC000D1FF58611A6942F040021A614FF4006157
:103AD000FFF798FF00F034F9FFF7B4FF2046BDE888
:103AE0001040FFF7CDBF002010BD00BF00200240F6
:103AF0002DE9F84312F00103144606D01F4B40F2A3
:103B0000F3221A600020BDE8F88385181C4A95420C
:103B100004D91A4A4FF43E711160F3E7FFF77CFFB6
:103B2000FFF770FFDFF86880451A4FF00109012C9C
:103B300005EB01060F4603D8FFF784FF0120E2E7FB
:103B40003B88C8F8109033800020FFF75BFFC8F86F
:103B50001000338831F8022B9BB29A420CD0074BED
:103B600040F20F321A60074B1E60074B1C60074B78
:103B70001F60FFF767FFC6E7023CD8E75C3A00200A
:103B800000000408503A0020583A0020543A00201F
:103B900000200240084908B50B7828B11BB9FFF78F
:103BA0003BFF01230B7008BD002BFCD0BDE8084093
:103BB0000870FFF747BF00BF603A002008B54FF418
:103BC00020414FF0005000F0BDF8BDE808404FF430
:103BD00000514FF0805000F0B5B800000846114683
:103BE00000F05EBE012000F05BBE0000084600F061
:103BF00075BE000030B583B0FFF71EFE0E4B0F4DB3
:103C0000DB692A684FF47A7101FB03F3934237BFF3
:103C10000B4A0B49516814682B602EBFD1E9004153
:103C2000013151601C1941F100010191FFF70EFEB5
:103C30000199204603B030BD20380020643A0020AE
:103C4000683A002030B583B0FFF7F6FD114B124DF6
:103C5000DB692A684FF47A7101FB03F3934237BFA3
:103C60000E4A0E49516814682B602EBFD1E90041FD
:103C7000013151601C1941F100010191FFF7E6FD8E
:103C800001994FF47A7200232046FCF791FA03B0B1
:103C900030BD00BF20380020643A0020683A002080
:103CA00010B50244064BD2B2904200D110BD441C64
:103CB00000B253F8200041F8040BE0B2F4E700BF73
:103CC000502800400F4B30B51C6A240407D41C6AEE
:103CD00044F440741C621C6A44F400441C620A4CA4
:103CE000236843F4807323600244084BD2B29042AD
:103CF00000D130BD441C00B251F8045B43F82050A1
:103D0000E0B2F4E70010024000700040502800408C
:103D100007B5012201A90020FFF7C2FF019803B0F7
:103D20005DF804FB13B50446FFF7F2FFA04205D08F
:103D3000012201A900200194FFF7C4FF02B010BDC9
:103D4000704700007047000070470000074B45F2C5
:103D500055521A6002225A6040F6FF729A604CF681
:103D6000CC421A60024B01221A70704700300040AA
:103D7000743A0020034B1B781BB1034B4AF6AA226E
:103D80001A607047743A002000300040044B1A68F3
:103D90002AB902F1804202F50432526A1A60704771
:103DA000703A0020024B4FF080725A62704700BF99
:103DB0000010024008B5FFF7E9FF024B1868C0F396
:103DC000407008BD703A002070470000FEE7000018
:103DD0000A4B0B480B4A90420BD30B4BDA1C121ABE
:103DE000C11E22F003028B4238BF00220021FDF7E2
:103DF000A5BA53F8041B40F8041BECE7F44B000889
:103E0000583C0020583C0020583C0020FEE70000B1
:103E100070B51B4B01630025044686B0586085626F
:103E20000E46FFF7E1FB04F11003C4E904334FF041
:103E3000FF33A361134BE561D969A5600A462B46A0
:103E4000C4E9082304F13401C4E900440E4AE562E0
:103E5000256580232046FFF709FD0123E0600B4A1A
:103E60000375009272680192B268CDE90223084B93
:103E70006846CDE90435FFF721FD06B070BD00BFEF
:103E8000483A002020380020904A0008954A00084F
:103E90000D3E00084B6843608B688360CB68C3604D
:103EA0000B6943614B6903628B6943620B68036072
:103EB0007047000008B51B4B9A6A42F4FC029A62F4
:103EC0009A6A22F4FC029A629A6A5A6942F4FC02E3
:103ED0005A61154A5B6911464FF09040FFF7DAFFCF
:103EE00002F11C0100F58060FFF7D4FF02F13801F8
:103EF00000F58060FFF7CEFF02F1540100F580600D
:103F0000FFF7C8FF02F1700100F58060FFF7C2FF04
:103F100002F18C0100F58060FFF7BCFFBDE80840AE
:103F200000F05AB8001002409C4A000808B500F0A2
:103F300093F9FFF759FCBDE80840FFF727BF0000E1
:103F40007047000010B5214CA36A63F4FC03A36220
:103F5000A36A03F4FC03A3624FF0FF32A36A236950
:103F600022612369002323612169E168E260E2683C
:103F7000E360E268E269164942F08052E261E26978
:103F80000A6842F480720A60226A02F44072B2F552
:103F9000407F1EBF4FF4803222622362236A1B04DB
:103FA00007D4236A43F440732362236A43F4004333
:103FB000236200F031F9A369064A43F00103A361CB
:103FC000A369136843F02003136010BD0010024082
:103FD00000700040000001401E4B1A6842F00102D0
:103FE0001A601A689007FCD55A6822F003025A60DA
:103FF0005A6812F00C02FBD1196801F0F90119603E
:104000005A601A6842F480321A601A689103FCD52B
:10401000114A5A604FF40452DA6230221A631A6865
:1040200042F080721A601A689201FCD50B49122284
:104030000A600A6802F00702022AFAD15A6842F0BE
:1040400002025A605A6802F00C02082AFAD11A6B6E
:104050001A6370470010024000241D000020024037
:10406000084A08B5516913680B4003F00103536116
:1040700023B1054A13680BB150689847BDE8084062
:10408000FFF7D6BA00040140783A0020084A08B584
:10409000516913680B4003F00203536123B1054AD1
:1040A00093680BB1D0689847BDE80840FFF7C0BAE5
:1040B00000040140783A0020084A08B551691368A5
:1040C0000B4003F00403536123B1054A13690BB19C
:1040D00050699847BDE80840FFF7AABA00040140BC
:1040E000783A0020084A08B5516913680B4003F07C
:1040F0000803536123B1054A93690BB1D06998470E
:10410000BDE80840FFF794BA00040140783A002067
:10411000084A08B5516913680B4003F01003536156
:1041200023B1054A136A0BB1506A9847BDE80840AD
:10413000FFF77EBA00040140783A0020174B10B513
:104140005A691C68144004F478725A61A30604D5B5
:10415000134A936A0BB1D06A9847600604D5104A97
:10416000136B0BB1506B9847210604D50C4A936B27
:104170000BB1D06B9847E20504D5094A136C0BB11B
:10418000506C9847A30504D5054A936C0BB1D06CCD
:104190009847BDE81040FFF74BBA00BF000401404C
:1041A000783A00201A4B10B55A691C68144004F480
:1041B0007C425A61620504D5164A136D0BB1506DED
:1041C0009847230504D5134A936D0BB1D06D9847DA
:1041D000E00404D50F4A136E0BB1506E9847A1044A
:1041E00004D50C4A936E0BB1D06E9847620404D587
:1041F000084A136F0BB1506F9847230404D5054A42
:10420000936F0BB1D06F9847BDE81040FFF710BA1D
:1042100000040140783A0020062108B50846FFF75F
:1042200031FA06210720FFF72DFA06210820FFF7B3
:1042300029FA06210920FFF725FA06210A20FFF7AF
:1042400021FA06211720FFF71DFABDE808400621D4
:104250002820FFF717BA000008B5FFF773FE00F03B
:1042600067F800F03DF8FFF76BFEBDE8084000F08E
:104270005DB80000026843681143016003B118474C
:1042800070470000143000F02FBA00004FF0FF33E9
:10429000143000F029BA0000383000F0A5BA000050
:1042A0004FF0FF33383000F09FBA0000143000F0B8
:1042B000F5B900004FF0FF31143000F0EFB9000005
:1042C000383000F04FBA00004FF0FF32383000F0C5
:1042D00049BA0000012914BF6FF013000020704795
:1042E00000F06CB8044B03600023C0E90233436064
:1042F00001230374704700BF444B000838B5C369FD
:1043000004460D461BB904210844FFF7B3FF2946B4
:1043100004F1140000F0A6F9002806DA201D4FF47D
:104320000061BDE83840FFF7A5BF38BD00F00EB80A
:104330000023054A19460133102BC2E9001102F18E
:104340000802F8D1704700BF783A00204FF0E02310
:10435000044A5A6100229A6107221A6108210B203F
:10436000FFF7A6B93F19010008B5302383F3118880
:10437000FFF760FA002383F3118808BD08B5FFF743
:10438000F3FFBDE80840FFF753B900000268436837
:104390001143016003B1184770470000024A1368D7
:1043A00043F0C0031360704700380140024A1368AD
:1043B00043F0C003136070470044004037B51D4C04
:1043C0001D4D2046FFF78EFF009404F114001B4999
:1043D0000023202200F038F92022009404F1380054
:1043E000174B184900F0B2F9174BC4E91735174CB1
:1043F0000C212520FFF746F92046FFF773FF04F153
:104400001400134900940023202200F01DF904F148
:104410003800104B10490094202200F097F90F4B00
:104420000C212620C4E9173503B0BDE83040FFF762
:1044300029B900BFF83A002000512502D03B0020E6
:104440009D430008103C002000380140643B0020E0
:10445000F03B0020AD430008303C00200044004009
:104460002DE9F047C66D3768F469346221070546C7
:1044700019D014F0080118BF4FF48071E20748BF4B
:1044800041F02001A30748BF41F04001600748BF49
:1044900041F08001302383F31188281DFFF776FF58
:1044A000002383F31188E2050AD5302383F31188B2
:1044B0004FF48061281DFFF769FF002383F3118803
:1044C0004FF030094FF0000A14F0200838D13B06B5
:1044D00016D54FF0300905F1380A200610D589F3BA
:1044E0001188504600F066F9002836DA0821281DA8
:1044F000FFF74CFF27F080033360002383F311881C
:10450000790614D5620612D5302383F31188D5E9D4
:1045100013239A4208D12B6C33B11021281D27F0A8
:104520004007FFF733FF3760002383F31188E3066A
:1045300019D5AA6E1369B3B1BDE8F04750691847A1
:1045400089F31188B38C95F8641028461940FFF759
:10455000D5FE8AF31188F469B6E780B2308588F316
:104560001188F469B9E7BDE8F087000008B5034891
:10457000FFF776FFBDE80840FFF75AB8F83A002089
:1045800008B50348FFF76CFFBDE80840FFF750B8D7
:10459000643B0020F8B5154682680669AA420B46BE
:1045A000816938BF8568761AB54204460BD2184631
:1045B0002A46FCF7B1FEA3692B44A361A3685B1BE9
:1045C000A3602846F8BD0CD918463246FCF7A4FE75
:1045D000AF1BE1683A463044FCF79EFEE3683B447B
:1045E000EBE718462A46FCF797FEE368E5E700008C
:1045F00083689342F7B51546044638BF8568D0E90D
:104600000460361AB5420BD22A46FCF785FE636970
:104610002B446361A36828465B1BA36003B0F0BD15
:104620000DD932460191FCF777FE0199E068AF1B86
:104630003A463144FCF770FEE3683B44E9E72A461A
:10464000FCF76AFEE368E4E710B50A440024C3619E
:10465000029B8460C0E90000C0E90511C1600261ED
:10466000036210BD08B5D0E90532934201D18268DA
:1046700082B98268013282605A1C42611970D0E9A5
:1046800004329A4224BFC36843610021FFF748F90E
:10469000002008BD4FF0FF30FBE7000070B530236D
:1046A00004460E4683F31188A568A5B1A368A269E4
:1046B000013BA360531CA36115782269934224BF78
:1046C000E368A361E3690BB120469847002383F3B5
:1046D0001188284607E031462046FFF711F90028E7
:1046E000E2DA85F3118870BD2DE9F74F04460E46D6
:1046F00017469846D0F81C904FF0300A8AF311887C
:104700004FF0000B154665B12A4631462046FFF7AB
:1047100041FF034660B941462046FFF7F1F8002803
:10472000F1D0002383F31188781B03B0BDE8F08F2C
:10473000B9F1000F03D001902046C847019B8BF3CD
:104740001188ED1A1E448AF31188DCE7C0E90511CF
:10475000C160C3611144009B8260C0E90000016137
:1047600003627047F8B504460D461646302383F3BE
:104770001188A768A7B1A368013BA36063695A1CAD
:1047800062611D70D4E904329A4224BFE368636118
:10479000E3690BB120469847002080F3118807E0B9
:1047A00031462046FFF7ACF80028E2DA87F311889B
:1047B000F8BD0000D0E905239A4210B501D1826806
:1047C0007AB98268013282605A1C82611C7803695E
:1047D0009A4224BFC36883610021FFF7A1F82046F5
:1047E00010BD4FF0FF30FBE72DE9F74F04460E46B2
:1047F00017469846D0F81C904FF0300A8AF311887B
:104800004FF0000B154665B12A4631462046FFF7AA
:10481000EFFE034660B941462046FFF771F80028D5
:10482000F1D0002383F31188781B03B0BDE8F08F2B
:10483000B9F1000F03D001902046C847019B8BF3CC
:104840001188ED1A1E448AF31188DCE70B460146F5
:10485000184600F02DB8000000F040B8012838BF1D
:10486000012010B50446204600F030F830B900F0C1
:1048700007F808B900F00CF88047F4E710BD000015
:10488000024B1868BFF35B8F704700BF503C00209D
:1048900008B5062000F084F80120FFF7ABF800000F
:1048A000024B0A4601461868FFF798B91811002014
:1048B00010B5054C13462CB10A4601460220AFF351
:1048C000008010BD2046FCE700000000024B0146BE
:1048D0001868FFF787B900BF18110020024B014686
:1048E0001868FFF783B900BF1811002010B501390F
:1048F0000244904201D1002005E0037811F8014FF5
:10490000A34201D0181B10BD0130F2E72DE9F041A0
:10491000A3B1C91A17780144044603F1FF3C8C4245
:10492000204601D9002009E00578BD4204F10104C8
:10493000F5D10CEB0405D618A54201D1BDE8F081F4
:1049400015F8018D16F801EDF045F5D0E7E7000008
:104950001F2938B504460D4604D9162303604FF0CD
:10496000FF3038BD426C12B152F821304BB92046AD
:1049700000F030F82A4601462046BDE8384000F0F5
:1049800017B8012B0AD0591C03D11623036001204C
:10499000E7E7002442F82540284698470020E0E752
:1049A000024B01461868FFF7D3BF00BF1811002063
:1049B00038B5074D00230446084611462B60FFF723
:1049C0001DF8431C02D12B6803B1236038BD00BF22
:1049D000543C0020FFF70CB8034611F8012B03F8F4
:1049E000012B002AF9D170476F72672E61726475CE
:1049F00070696C6F742E663330332D4D6174656B46
:104A00004750530040A2E4F1646891060041A3E5D9
:104A1000F2656992070000004261642043414E49FB
:104A20006661636520696E6465782E008000000011
:104A30000080000000008000000000000000000076
:104A40003D1B000821230008812200084D1B00089F
:104A5000811B00087D1D0008511B0008611B000818
:104A6000551B00085D1B0008591B0008A51C000809
:104A7000651B0008ED250008751B0008791C00085F
:104A800063300000804A000878380020483A00204F
:104A90006D61696E0069646C65000000A001A82A60
:104AA00000000000FAAABEAA50001424EFFF000084
:104AB00000770000709709000000A00000000000CF
:104AC000AAAAFAAA00005000FFFF000000000000A0
:104AD000007700000000000000000000AAAAAAAAB7
:104AE00000000000FFFF00000000000000000000C8
:104AF0000000000000000000AAAAAAAA000000000E
:104B0000FFFF0000000000000000000000000000A7
:104B100000000000AAAAAAAA00000000FFFF0000EF
:104B20000000000000000000000000000000000085
:104B3000AAAAAAAA00000000FFFF000000000000CF
:104B40000000000000000000A14200088D420008A3
:104B5000C9420008B5420008C1420008AD42000841
:104B60009942000885420008D542000874B6FF7FCC
:104B70000100000000000000EC0300000000000045
:104B80000098030000000000FE2A0100D20400008B
:104B90001C110020000000000000000000000000C8
:104BA0000000000000000000000000000000000005
:104BB00000000000000000000000000000000000F5
:104BC00000000000000000000000000000000000E5
:104BD00000000000000000000000000000000000D5
:104BE00000000000000000000000000000000000C5
:044BF00000000000C1
:00000001FF
